:020000040000FA
:100000008316D0308100003086001F3085008312B7
:1000100000000000000000000000000000000000E0
:10002000860185010614051C1B28851C2A284220F0
:100030000610422012280A30A30086010614051873
:100040001228851C39287B20061006117F20A30B5F
:100050001D28BD280A30A300860106148518122821
:10006000051C39285D20061086119620A30B2C282C
:10007000B82806140611861186140518B8288518A4
:10008000BD2839280530A000FF30A100FF30A200B4
:10009000A20B4828A10B4628A00B08000530A000A1
:1000A000FF30A100FF30A200A20B5428851C392884
:1000B000AD20A10B5228A00B080061206120612017
:1000C00008000530A000FF30A100FF30A200A20B05
:1000D0006728051C39287020A10B6528A00B080093
:1000E0008611061186157720861177200800810178
:1000F000811F782808004E204E204E2008008820BE
:10010000882088208820882088208820882008004F
:100110000530A000FF30A100FF30A200A20B8E2806
:10012000851C3928A10B8C28A00B08009F209F203C
:100130009F209F209F209F209F209F200800053008
:10014000A000FF30A100FF30A200A20BA528051CD3
:100150003928A10BA328A00B08008611061106154B
:10016000B4200611B42008008101811FB5280800C1
:100170008601850185180828B8288601850105189B
:040180000828BD2866
:02400E00F13F80
:00000001FF
